:020000040800F2
:1000000000060020E1020008E3020008E302000805
:10001000E3020008E3020008E3020008E30200082C
:10002000E3020008E3020008E302000819320008B6
:10003000E3020008E3020008E3020008E30200080C
:10004000E3020008E3020008E3020008E3020008FC
:10005000E3020008E3020008E3020008E3020008EC
:10006000E3020008E3020008E3020008C1110008EF
:10007000E911000815120008411200086D1200086D
:1000800095120008C1120008E3020008E30200080C
:10009000E3020008E3020008E3020008E3020008AC
:1000A000E3020008E3020008E3020008E30200089C
:1000B0001D4A0008E3020008E3020008E30200080A
:1000C000E3020008E3020008E3020008E30200087C
:1000D000E3020008E3020008E3020008E30200086C
:1000E000E3020008E3020008E3020008E30200085C
:1000F000E3020008E3020008E3020008ED12000832
:10010000E3020008F5490008E3020008E3020008E2
:10011000E3020008E3020008E3020008E30200082B
:1001200019130008411300086D1300089913000803
:10013000C5130008E3020008E3020008E302000818
:10014000E3020008E3020008E3020008E3020008FB
:10015000ED1300081914000845140008E302000814
:10016000E3020008E3020008E3020008E3020008DB
:10017000E3020008053E0008E3020008E30200086D
:10018000E3020008E3020008094A0008E30200084D
:10019000E3020008E3020008E3020008E3020008AB
:1001A000E3020008E3020008E3020008E30200089B
:1001B000E3020008E3020008E3020008E30200088B
:1001C000E3020008E3020008E3020008E30200087B
:1001D000E3020008F13D0008E3020008E302000822
:1001E000E3020008E3020008E3020008E30200085B
:1001F000E3020008E3020008E3020008E30200084B
:10020000E3020008E3020008E3020008E30200083A
:10021000E3020008E3020008E3020008E30200082A
:10022000E3020008E3020008E3020008E30200081A
:10023000E3020008E3020008E3020008E30200080A
:10024000E3020008E3020008E3020008E3020008FA
:10025000E3020008E3020008E3020008E3020008EA
:10026000E3020008E3020008E3020008E3020008DA
:10027000E3020008E3020008E3020008E3020008CA
:10028000E3020008E3020008E3020008E3020008BA
:10029000E3020008E3020008E3020008E3020008AA
:1002A000E3020008E3020008E3020008E30200089A
:1002B000E3020008E3020008E3020008E30200088A
:1002C000E3020008E3020008E3020008E30200087A
:1002D000E3020008E3020008E3020008E30200086A
:1002E00002E000F000F8FEE772B6374880F30888B5
:1002F000364880F3098836483649086040F20000E5
:10030000CCF200004EF63471CEF200010860BFF36B
:100310004F8FBFF36F8F40F20000C0F2F0004EF637
:100320008851CEF200010860BFF34F8FBFF36F8F8B
:100330004FF00000E1EE100A4EF63C71CEF20001E3
:100340000860062080F31488BFF36F8F02F0C6FFA9
:1003500004F008F94FF055301F491B4A91423CBF49
:1003600041F8040BFAE71D49184A91423CBF41F895
:10037000040BFAE71A491B4A1B4B9A423EBF51F83D
:10038000040B42F8040BF8E700201849184A914280
:100390003CBF41F8040BFAE702F0DEFF04F066F917
:1003A000144C154DAC4203DA54F8041B8847F9E7A6
:1003B00000F042F8114C124DAC4203DA54F8041B21
:1003C0008847F9E702F0C6BF00060020002200209F
:1003D0000000000808ED00E00000002000060020FA
:1003E000D85A000800220020642200206822002041
:1003F000E44A0020E0020008E0020008E0020008F1
:10040000E00200082DE9F04F2DED108AC1F80CD064
:10041000D0F80CD0BDEC108ABDE8F08F002383F338
:1004200011882846A047002002F05EF9FEE702F09E
:10043000E3F800DFFEE7000038B500F04DFC00F007
:1004400011FE02F093FE054602F0D8FE0446C0B944
:100450000E4B9D4217D001339D4241F2883512BFA9
:10046000044600250124002002F08AFE0CB100F0B1
:1004700073F800F095FD284600F01CF900F06CF8C8
:10048000F9E70025EFE70546EDE700BF010007B0FB
:1004900008B500F0EDFBA0F120035842584108BD1B
:1004A00007B5042101900DEB010000F0FFFB03B044
:1004B0005DF804FB38B5302383F3118817480368CF
:1004C0000BB102F0F5F90023154A4FF47A71134885
:1004D00002F0E4F9002383F31188124C236813B16E
:1004E0002368013B2360636813B16368013B636069
:1004F0000D4D2B7833B963687BB9022000F0B2FC54
:10050000322363602B78032B07D163682BB9022059
:1005100000F0A8FC4FF47A73636038BD68220020B5
:10052000B50400088823002080220020084B1870A2
:1005300003280CD8DFE800F008050208022000F0CC
:1005400083BC022000F070BC024B00225A6070474E
:100550008022002088230020F8B5504B504A1C46CA
:100560001968013100F0998004339342F8D1626830
:100570004C4B9A4240F291804B4B9B6803F10063D5
:1005800003F500339A4280F08880002000F0BEFB23
:100590000220FFF7CBFF454B0021D3F8E820C3F83A
:1005A000E810D3F81021C3F81011D3F81021D3F8B4
:1005B000EC20C3F8EC10D3F81421C3F81411D3F8CD
:1005C0001421D3F8F020C3F8F010D3F81821C3F8A1
:1005D0001811D3F81821D3F8802042F00062C3F834
:1005E0008020D3F8802022F00062C3F88020D3F866
:1005F0008020D3F8802042F00072C3F88020D3F826
:10060000802022F00072C3F88020D3F8803072B6C8
:100610004FF0E023C3F8084DD4E90004BFF34F8F37
:10062000BFF36F8F224AC2F88410BFF34F8F536914
:1006300023F480335361BFF34F8FD2F8803043F6F9
:10064000E076C3F3C905C3F34E335B0103EA060C3E
:1006500029464CEA81770139C2F87472F9D2203BFD
:1006600013F1200FF2D1BFF34F8FBFF36F8FBFF3A2
:100670004F8FBFF36F8F536923F40033536100230F
:10068000C2F85032BFF34F8FBFF36F8F302383F325
:100690001188854680F308882047F8BD00000208CD
:1006A00020000208FFFF0108002200200044025839
:1006B00000ED00E02DE9F04F95B0DFF8D892202250
:1006C000FF21029004A8D9F8085000F013FCA84AB2
:1006D0001378A3B90121A74811700360302383F375
:1006E000118803680BB102F0E3F80023A24A4FF42B
:1006F0007A71A04802F0D2F8002383F31188029B9C
:1007000013B19E4B029A1A609D4A1378032B03D0B3
:1007100000231370994A53604FF0000B029C5E4611
:10072000DA46CDF804B0012000F08EFB24B1934BE3
:100730001B68002B00F02882002000F099FAB0F12D
:100740000008F3DB012000F06FFBA8F121031F2B51
:10075000E9D801A252F823F0D9070008F5070008EC
:100760008308000827070008270700082707000854
:100770000D090008FF0A0008F10900084D0A0008E9
:10078000730A0008990A000827070008AB0A000846
:10079000CF0A0008470B0008610800082707000877
:1007A0008F0B0008E507000861080008270700080C
:1007B0004D0A000827070008270700082707000838
:1007C0002707000827070008270700082707000851
:1007D00027070008830800080220FFF759FE0028B9
:1007E00040F0FF81029B02216648BBF1000F08BF69
:1007F0001C4640E04FF47A7000F03AFA071EF1DB35
:100800000220FFF745FE0028ECD0013F052F00F243
:10081000EA81DFE807F003070A0D10330520FFF730
:100820003FFE14E0D9F80000F9E7D9F80400F6E734
:10083000D9F80800F3E74FF01C08404608F1040817
:1008400000F066FAFFF72CFEB8F12C0FF5D101206D
:10085000019B4FF0000A00FA07F71F43FBB2019318
:1008600000F094FB2EB1019B03F00B030B2B08BF90
:1008700000240221444800F019FA54E7D9F80C008A
:10088000CDE7002EAED0019B03F00B030B2BA9D1BB
:100890000220FFF7FDFD07460028A3D00120002617
:1008A00000F034FA0220FFF741FE1FFA86FB58469B
:1008B00000F03CFA044688B1A8F1400258460136DF
:1008C0005142514100F042FA0028EED1BB460446A5
:1008D00002212E483E4600F0E9F924E72546012092
:1008E000FFF724FED9F80830AB4207D9284600F0BC
:1008F0000FFA013040F07A810435F3E70025204BF0
:10090000BB463E461D701D4B5D60A9E7002E3FF4BF
:1009100069AF019B03F00B030B2B7FF463AF022045
:10092000FFF704FE322000F0A3F9B0F10008FFF653
:1009300059AF18F003077FF455AF08EB0503D9F85A
:10094000082093423FF64EAFB8F5807F3FF74AAF9D
:100950000F4BB84503931FDD4FF47A7000F088F910
:100960000028FFF63FAF039B013703F8010BF0E7C8
:100970008423002068220020B5040008882300207A
:1009800080220020145600080C560008105600085B
:100990008422002000220020C820FFF779FD0746AE
:1009A00000283FF41FAF1F2D11D8C5F1200204AB62
:1009B00025F003008F494245184428BF4246039260
:1009C00000F072FA039AFF218A4800F093FA4FEA86
:1009D000A803C8F3870287492846039300F092FAD8
:1009E000064600283FF474AF039B05EB830537E709
:1009F0000220FFF74DFD00283FF4F4AE00F0C4F9EB
:100A000000283FF4EFAE0027B846D9F80830BB42C3
:100A100018D91F2F11D8049B01330ED027F00303E0
:100A200014AA134453F8403C0C93404604220CA9EA
:100A3000043700F0AFFB8046E7E7384600F068F97E
:100A40000C90F2E74046FFF72BFD09E700236421F5
:100A50000CA80C9300F020F900287FF4C3AE02200C
:100A6000FFF716FD00283FF4BDAE0C9800F082F9A8
:100A7000E9E7002364210CA80C9300F00DF900288D
:100A80007FF4B0AE0220FFF703FD00283FF4AAAECA
:100A90000C9800F071F9D6E70220FFF7F9FC002866
:100AA0003FF4A0AE00F080F9CDE70220FFF7F0FCA4
:100AB00000283FF497AE0CA9142000F07BF90390B6
:100AC000FFF7EEFC03990CA800F0F0F8C8E602204E
:100AD000FFF7DEFC00283FF485AE474B0CAF03F177
:100AE000100C1868083353F8041C3A46634503C2D7
:100AF0001746F6D11020FFF7D3FC1021E3E7322090
:100B000000F0B6F8071EFFF66DAEBB077FF46AAEC5
:100B100007EB0A03D9F8082093423FF663AE0220A0
:100B2000FFF7B6FC00283FF45DAE27F003075744FB
:100B3000BA453FF495AE50460AF1040A00F0E8F8D1
:100B4000FFF7AEFCF4E74FF47A70FFF7A1FC002842
:100B50003FF448AE00F018F9002849D0049B013357
:100B60000BD0082204A9002000F0CCF900283FD0C7
:100B70002022FF2104A800F0BDF92048022100F046
:100B800095F81F4801F0B6FD15B0BDE8F08F002EB6
:100B90003FF428AE019B03F00B030B2B7FF422AE36
:100BA000002364210CA80C9300F076F80746002877
:100BB0007FF418AE0220FFF76BFC804600283FF45C
:100BC00011AE02210D4800F071F841F2883001F0B9
:100BD00091FD0C9800F024FA46463C4600F0D6F908
:100BE000A1E506463CE64FF0000AFBE5BB466FE692
:100BF00037466DE684220020F85500080C560008A0
:100C0000A08601002DE9F84F4FF47A7306460D4691
:100C1000002402FB03F7DFF85080DFF8509098F9CA
:100C200000305FFA84FA5A1C01D0A34212D159F85D
:100C300024002A4631460368D3F820B03B46D84703
:100C4000854207D1074B012083F800A0BDE8F88F4B
:100C50000124E4E7002CFBD04FF4FA7001F04AFDC8
:100C60000020F3E7D42300201022002014220020CB
:100C7000002307B5024601210DF107008DF807306A
:100C8000FFF7C0FF20B19DF8070003B05DF804FB3B
:100C90004FF0FF30F9E700000A46042108B5FFF7DE
:100CA000B1FF80F00100C0B2404208BD074B0A46C8
:100CB00030B41978064B53F821400146236820468A
:100CC000DD69044BAC4630BC604700BFD423002034
:100CD00014220020A086010070B50A4E00240A4D9F
:100CE00002F03CF8308028683388834208D902F04B
:100CF00031F82B6804440133B4F5003F2B60F2D384
:100D000070BD00BFD62300209023002002F000B960
:100D100000F1006000F500300068704700F10060ED
:100D2000920000F5003002F075B80000054B1A681B
:100D3000054B1B889B1A834202D9104402F00AB863
:100D40000020704790230020D623002038B50446A9
:100D5000074D29B128682044BDE8384002F012B898
:100D60002868204401F0FCFF0028F3D038BD00BF04
:100D7000902300200020704700F1FF5000F58F10F5
:100D8000D0F8000870470000064991F8243033B1CC
:100D900000230822086A81F82430FFF7BFBF012032
:100DA000704700BF94230020014B1868704700BFB4
:100DB0000010005C194B01380322084470B51D680F
:100DC000174BC5F30B042D0C1E88A6420BD15C6893
:100DD0000A46013C824213460FD214F9016F4EB10C
:100DE00002F8016BF6E7013A03F10803ECD1814206
:100DF0000B4602D22C2203F8012B0424094A168840
:100E0000AE4204D1984284BF967803F8016B013C4E
:100E100002F10402F3D1581A70BD00BF0010005C4B
:100E20001C22002044560008022804D1054B4FF430
:100E300080029A6170470128FCD1024B4FF40002F6
:100E4000F7E700BF00200258022803D1044B4022DC
:100E50009A6170470128FCD1014B8022F8E700BF5E
:100E600000200258022805D1064A536983F0400346
:100E7000536170470128FCD1024A536983F0800313
:100E8000F6E700BF0020025870B504464FF47A76AA
:100E90004CB1412C254628BF412506FB05F0641BBB
:100EA00001F028FCF4E770BD002310B5934203D095
:100EB000CC5CC4540133F9E710BD0000013810B513
:100EC00010F9013F3BB191F900409C4203D11AB1A6
:100ED0000131013AF4E71AB191F90020981A10BDD6
:100EE0001046FCE703460246D01A12F9011B0029FE
:100EF000FAD1704702440346934202D003F8011B23
:100F0000FAE770472DE9F8431F4D14460746884617
:100F100095F8242052BBDFF870909CB395F82430EC
:100F20002BB92022FF2148462F62FFF7E3FF95F8F7
:100F300024004146C0F1080205EB8000A24228BF10
:100F40002246D6B29200FFF7AFFF95F82430A41BDB
:100F500017441E449044E4B2F6B2082E85F824608B
:100F6000DBD1FFF711FF0028D7D108E02B6A03EB94
:100F700082038342CFD0FFF707FF0028CBD10020A8
:100F8000BDE8F8830120FBE794230020024B1A7888
:100F9000024B1A70704700BFD4230020102200209B
:100FA00038B51A4C1A4D204600F0BEFE29462046A0
:100FB00000F0E6FE2D684FF47A70D5F89020D2F854
:100FC000043843F00203C2F80438FFF75DFF11490B
:100FD000284600F0E3FFD5F890200F4DD2F80438F2
:100FE000286823F002030D49A042C2F804384FF4E8
:100FF000E1330B6001D000F0F5FD6868A04204D039
:101000000649BDE8384000F0EDBD38BD382B002062
:10101000405800084858000814220020BC23002033
:101020000C4B70B50C4D04461E780C4B55F8262021
:101030009A420DD00A4B002118221846FFF75AFF9A
:101040000460014655F82600BDE8704000F0CABDB6
:1010500070BD00BFD423002014220020382B0020B4
:10106000BC2300202DE9F04771B6464B01201D68D6
:10107000454BB3F8008000231A46194600F08AFA5F
:101080000446802001F0E2FF0746002862D0002CD1
:1010900060D03E4EADB24FF0800A7369284643F0EF
:1010A000C0637361D6F8143143F0C063C6F81431DD
:1010B00001F050FE05EB080200FB05F34FF4D06C85
:1010C00050434FF03D0E984233D93269520144D417
:1010D000D6F81021510140D4216803F100628A60E2
:1010E0002268D7602268C2F804A02268C2F800C053
:1010F000D4F80090D9F8002042F00102C9F800208D
:10110000D4F80090D9F8002022F01E02C9F800207F
:10111000D4F80090D9F80020D207FBD494F80C90B2
:10112000803361680EFA09F20A60CCE7002001F012
:10113000EFFE204600F06EFA384601F0C1FF134B77
:101140005A6942F0C0625A61D3F8142142F0C06279
:10115000C3F8142161B6BDE8F0870D4B9A6A42F4DA
:1011600000729A629A6A42F400429A6261B600265C
:10117000012001F0CDFEB045D8D9A819013601F003
:1011800001FEF8E790230020D62300200020005223
:1011900000ED00E030B50A44084D91420DD011F841
:1011A000013B5840082340F30004013B2C4013F05E
:1011B000FF0384EA5000F6D1EFE730BD2083B8ED9D
:1011C00008B5074B074A196801F03D01996053685B
:1011D0000BB190689847BDE8084002F055B800BFD1
:1011E00000000240D823002008B5084B196889097F
:1011F00001F03D018A019A60054AD3680BB110697C
:101200009847BDE8084002F03FB800BF0000024028
:10121000D823002008B5084B1968090C01F03D01DE
:101220000A049A60054A53690BB190699847BDE872
:10123000084002F029B800BF00000240D823002077
:1012400008B5084B1968890D01F03D018A059A60BF
:10125000054AD3690BB1106A9847BDE8084002F00F
:1012600013B800BF00000240D823002008B5074B88
:10127000074A596801F03D01D960536A0BB1906A81
:101280009847BDE8084001F0FFBF00BF00000240E2
:10129000D823002008B5084B5968890901F03D01A1
:1012A0008A01DA60054AD36A0BB1106B9847BDE832
:1012B000084001F0E9BF00BF00000240D823002031
:1012C00008B5084B5968090C01F03D010A04DA60C1
:1012D000054A536B0BB1906B9847BDE8084001F08D
:1012E000D3BF00BF00000240D823002008B5084B40
:1012F0005968890D01F03D018A05DA60054AD36B12
:101300000BB1106C9847BDE8084001F0BDBF00BFAD
:1013100000000240D823002008B5074B074A19688F
:1013200001F03D019960536C0BB1906C9847BDE89A
:10133000084001F0A9BF00BF00040240D8230020EC
:1013400008B5084B1968890901F03D018A019A60C6
:10135000054AD36C0BB1106D9847BDE8084001F009
:1013600093BF00BF00040240D823002008B5084BFB
:101370001968090C01F03D010A049A60054A536D91
:101380000BB1906D9847BDE8084001F07DBF00BFEC
:1013900000040240D823002008B5084B1968890DC5
:1013A00001F03D018A059A60054AD36D0BB1106EBC
:1013B0009847BDE8084001F067BF00BF0004024045
:1013C000D823002008B5074B074A596801F03D01B2
:1013D000D960536E0BB1906E9847BDE8084001F09C
:1013E00053BF00BF00040240D823002008B5084BBB
:1013F0005968890901F03D018A01DA60054AD36E16
:101400000BB1106F9847BDE8084001F03DBF00BF29
:1014100000040240D823002008B5084B5968090C85
:1014200001F03D010A04DA60054A536F0BB1906F79
:101430009847BDE8084001F027BF00BF0004024004
:10144000D823002008B5084B5968890D01F03D01EB
:101450008A05DA60054AD36F13B1D2F88000984745
:10146000BDE8084001F010BF00040240D82300206E
:1014700000230C4910B51A460B4C0B6054F823009E
:10148000026001EB430004334260402BF6D1074A6F
:101490004FF0FF339360D360C2F80834C2F80C34C5
:1014A00010BD00BFD82300205456000800000240A1
:1014B0000F28F8B510D9102810D0112811D01228F3
:1014C00008D10F240720DFF8C8E00126DEF800501D
:1014D000A04208D9002653E00446F4E70F24002078
:1014E000F1E70724FBE706FA00F73D424AD1264C14
:1014F0004FEA001C3D4304EB00160EEBC000CEF893
:101500000050C0E90123FBB273B12048D0F8D830B5
:1015100043F00103C0F8D830D0F8003143F00103A4
:10152000C0F80031D0F8003117F47F4F0ED01748C3
:10153000D0F8D83043F00203C0F8D830D0F80031EA
:1015400043F00203C0F80031D0F8003154F80C0029
:10155000036823F01F030360056815F00105FBD144
:1015600004EB0C033D2493F80CC05F6804FA0CF400
:101570003C6021240560446112B1987B00F066F95B
:101580003046F8BD0130A3E7545600080044025825
:10159000D823002010B5302484F31188FFF788FF8A
:1015A000002383F3118810BD10B50446807B00F042
:1015B00063F901231549627B03FA02F20B6823EAFF
:1015C0000203DAB20B6072B9114AD2F8D81021F0D6
:1015D0000101C2F8D810D2F8001121F00101C2F8BF
:1015E0000011D2F8002113F47F4F0ED1084BD3F82D
:1015F000D82022F00202C3F8D820D3F8002122F02C
:101600000202C3F80021D3F8003110BDD823002016
:101610000044025808B5302383F31188FFF7C4FF54
:10162000002383F3118808BD0268436811430160F9
:1016300003B1184770470000024A136843F0C00323
:10164000136070470078004013B50E4C204600F040
:10165000BDFA04F1140000234FF400720A4900940B
:1016600000F07AF9094B4FF40072094904F138008F
:10167000009400F0F3F9074A074BC4E9172302B0BE
:1016800010BD00BF5C240020C824002039160008CB
:10169000C82600200078004000E1F505037C30B545
:1016A000244C002918BF0C46012B11D1224B984223
:1016B0000ED1224BD3F8E82042F08042C3F8E82054
:1016C000D3F8102142F08042C3F81021D3F8103132
:1016D0002268036EC16D03EB52038466B3FBF2F321
:1016E0006268150442BF23F0070503F0070343EACD
:1016F0004503CB60A36843F040034B60E36843F0CD
:1017000001038B6042F4967343F001030B604FF0CA
:10171000FF330B62510505D512F0102205D0B2F14E
:10172000805F04D080F8643030BD7F23FAE73F2328
:10173000F8E700BF545700085C240020004402581A
:101740002DE9F047C66D05463768F4692107346214
:101750001AD014F0080118BF4FF48071E20748BF97
:1017600041F02001A3074FF0300348BF41F0400192
:10177000600748BF41F0800183F31188281DFFF7FF
:1017800053FF002383F31188E2050AD5302383F346
:1017900011884FF48061281DFFF746FF002383F373
:1017A00011884FF030094FF0000A14F0200838D1AA
:1017B0003B0616D54FF0300905F1380A200610D542
:1017C00089F31188504600F07DF9002836DA0821A7
:1017D000281DFFF729FF27F080033360002383F3E0
:1017E0001188790614D5620612D5302383F3118847
:1017F000D5E913239A4208D12B6C33B127F0400767
:101800001021281DFFF710FF3760002383F3118894
:10181000E30618D5AA6E1369ABB15069BDE8F0476D
:10182000184789F31188736A284695F8641019409F
:1018300000F0E6F98AF31188F469B6E7B06288F33C
:101840001188F469BAE7BDE8F0870000090100F1EA
:101850006043012203F56143C9B283F8001300F02D
:101860001F039A4043099B0003F1604303F5614362
:10187000C3F880211A60704700F01F0301229A40CC
:10188000430900F160409B0000F5614003F16043B3
:1018900003F56143C3F88020C3F88021002380F85A
:1018A00000337047F8B51546826804460B46AA42D5
:1018B00000D28568A1692669761AB5420BD218460E
:1018C0002A46FFF7F1FAA3692B44A3612846A368CF
:1018D0005B1BA360F8BD0CD9AF1B18463246FFF75F
:1018E000E3FA3A46E1683044FFF7DEFAE3683B4446
:1018F000EBE718462A46FFF7D7FAE368E5E700006A
:1019000083689342F7B50446154600D28568D4E94A
:101910000460361AB5420BD22A46FFF7C5FA63694E
:101920002B4463612846A3685B1BA36003B0F0BD32
:101930000DD93246AF1B0191FFF7B6FA01993A462D
:10194000E0683144FFF7B0FAE3683B44E9E72A4630
:10195000FFF7AAFAE368E4E710B50A440024C3617C
:10196000029B8460C16002610362C0E90000C0E9BB
:10197000051110BD08B5D0E90532934201D1826846
:1019800082B98268013282605A1C4261197000215A
:10199000D0E904329A4224BFC368436100F0DEFEFE
:1019A000002008BD4FF0FF30FBE7000070B530238A
:1019B00004460E4683F31188A568A5B1A368A26901
:1019C000013BA360531CA36115782269934224BF95
:1019D000E368A361E3690BB120469847002383F3D2
:1019E0001188284607E03146204600F0A7FE00286F
:1019F000E2DA85F3118870BD2DE9F74F04460E46F3
:101A000017469846D0F81C904FF0300A8AF3118898
:101A10004FF0000B154665B12A4631462046FFF7C8
:101A200041FF034660B94146204600F087FE00288A
:101A3000F1D0002383F31188781B03B0BDE8F08F49
:101A4000B9F1000F03D001902046C847019B8BF3EA
:101A50001188ED1A1E448AF31188DCE7C160C36166
:101A6000009B82600362C0E905111144C0E90000D7
:101A700001617047F8B504460D461646302383F3DE
:101A80001188A768A7B1A368013BA36063695A1CCA
:101A900062611D70D4E904329A4224BFE368636135
:101AA000E3690BB120469847002080F3118807E0D6
:101AB0003146204600F042FE0028E2DA87F3118822
:101AC000F8BD0000D0E9052310B59A4201D1826823
:101AD0007AB982680021013282605A1C82611C78C6
:101AE00003699A4224BFC368836100F037FE204631
:101AF00010BD4FF0FF30FBE72DE9F74F04460E46CF
:101B000017469846D0F81C904FF0300A8AF3118897
:101B10004FF0000B154665B12A4631462046FFF7C7
:101B2000EFFE034660B94146204600F007FE00285C
:101B3000F1D0002383F31188781B03B0BDE8F08F48
:101B4000B9F1000F03D001902046C847019B8BF3E9
:101B50001188ED1A1E448AF31188DCE70268436895
:101B60001143016003B11847704700001430FFF7BC
:101B700043BF00004FF0FF331430FFF73DBF0000BC
:101B80003830FFF7B9BF00004FF0FF333830FFF7B0
:101B9000B3BF00001430FFF709BF00004FF0FF3162
:101BA0001430FFF703BF00003830FFF763BF0000B9
:101BB0004FF0FF323830FFF75DBF0000012914BF3E
:101BC0006FF0130000207047FFF73EBD044B036029
:101BD00000234360C0E9023301230374704700BF50
:101BE0006C57000810B53023044683F31188FFF7C3
:101BF00055FD02230020237480F3118810BD0000DE
:101C000038B5C36904460D461BB904210844FFF7E3
:101C1000A5FF294604F11400FFF7ACFE002806DA00
:101C2000201D4FF40061BDE83840FFF797BF38BD75
:101C3000026843681143016003B118477047000010
:101C400013B5406B00F58054D4F8A4381A681178A5
:101C5000042914D1017C022911D119790123128997
:101C60008B4013420BD101A94C3002F0FDF9D4F89E
:101C7000A4480246019B2179206800F0DFF902B0F8
:101C800010BD0000143002F07FB900004FF0FF33A8
:101C9000143002F079B900004C3002F051BA000063
:101CA0004FF0FF334C3002F04BBA0000143002F01A
:101CB0004DB900004FF0FF31143002F047B9000079
:101CC0004C3002F01DBA00004FF0FF324C3002F0F1
:101CD00017BA00000020704710B500F58054D4F802
:101CE000A4381A681178042917D1017C022914D16B
:101CF0005979012352898B4013420ED1143002F0DE
:101D0000DFF8024648B1D4F8A4484FF44073617933
:101D10002068BDE8104000F07FB910BD406BFFF7B0
:101D2000DBBF0000704700007FB5124B0125042681
:101D3000044603600023057400F1840243602946D1
:101D4000C0E902330C4B0290143001934FF44073FE
:101D5000009602F091F8094B04F69442294604F1EA
:101D60004C000294CDE900634FF4407302F058F93F
:101D700004B070BD945700081D1D0008411C0008E8
:101D80000A68302383F311880B790B3342F8230060
:101D90004B79133342F823008B7913B10B3342F89C
:101DA000230000F58053C3F8A41802230374002015
:101DB00080F311887047000038B5037F044613B1E3
:101DC00090F85430ABB90125201D0221FFF730FFF8
:101DD00004F114006FF00101257700F0CBFC04F151
:101DE0004C0084F854506FF00101BDE8384000F019
:101DF000C1BC38BD10B5012104460430FFF718FFFF
:101E00000023237784F8543010BD000038B5044611
:101E10000025143002F048F804F14C00257702F058
:101E200017F9201D84F854500121FFF701FF2046C7
:101E3000BDE83840FFF750BF90F8803003F06003F2
:101E4000202B06D190F881200023212A03D81F2AB5
:101E500006D800207047222AFBD1C0E91D3303E0D9
:101E6000034A426707228267C3670120704700BFA9
:101E70003422002037B500F58055D5F8A4381A680B
:101E8000117804291AD1017C022917D1197901236B
:101E900012898B40134211D100F14C04204602F00C
:101EA00097F958B101A9204602F0DEF8D5F8A44808
:101EB0000246019B2179206800F0C0F803B030BDD4
:101EC00001F10B03F0B550F8236085B004460D46D0
:101ED000FEB1302383F3118804EB8507301D082100
:101EE000FFF7A6FEFB6806F14C005B691B681BB19F
:101EF000019002F0C7F8019803A902F0B5F8024674
:101F000048B1039B2946204600F098F8002383F34C
:101F1000118805B0F0BDFB685A691268002AF5D037
:101F20001B8A013B1340F1D104F18002EAE7000073
:101F3000133138B550F82140ECB1302383F31188C8
:101F400004F58053D3F8A4281368527903EB820375
:101F5000DB689B695D6845B104216018FFF768FE86
:101F6000294604F1140001F0B5FF2046FFF7B4FE46
:101F7000002383F3118838BD7047000001F082BA56
:101F800001234022002110B5044600F8303BFEF743
:101F9000B1FF0023C4E9013310BD000010B53023A8
:101FA000044683F311882422416000210C30FEF79F
:101FB000A1FF204601F088FA02230020237080F35D
:101FC000118810BD70B500EB8103054650690E46BF
:101FD0001446DA6018B110220021FEF78BFFA069C9
:101FE00018B110220021FEF785FF31462846BDE8D2
:101FF000704001F06FBB000083682022002103F0D5
:10200000011310B5044683601030FEF773FF2046BD
:10201000BDE8104001F0EABBF0B4012500EB8104FB
:1020200047898D40E4683D43A469458123600023CE
:10203000A2606360F0BC01F007BC0000F0B40125B1
:1020400000EB810407898D40E4683D4364690581A4
:1020500023600023A2606360F0BC01F07DBC00003F
:1020600070B5022300250446242203702946C0F8D7
:1020700088500C3040F8045CFEF73CFF204684F8A2
:10208000705001F0BBFA63681B6823B129462046F3
:10209000BDE87040184770BD0378052B10B50446A5
:1020A0000AD080F88C300523037043681B680BB19D
:1020B000042198470023A36010BD00000178052982
:1020C00006D190F88C20436802701B6803B1184752
:1020D0007047000070B590F87030044613B10023CB
:1020E00080F8703004F18002204601F0A3FB6368A1
:1020F0009B68B3B994F8803013F0600535D00021A7
:10210000204601F095FE0021204601F085FE63681F
:102110001B6813B1062120469847062384F87030C7
:1021200070BD204698470028E4D0B4F88630A26FEE
:102130009A4288BFA36794F98030A56F002B4FF0B7
:10214000300380F20381002D00F0F280092284F830
:10215000702083F3118800212046D4E91D23FFF766
:102160006DFF002383F31188DAE794F8812003F0F0
:102170007F0343EA022340F20232934200F0C5801B
:1021800021D8B3F5807F48D00DD8012B3FD0022B4A
:1021900000F09380002BB2D104F188026267022222
:1021A000A267E367C1E7B3F5817F00F09B80B3F5D9
:1021B000407FA4D194F88230012BA0D1B4F88830AC
:1021C00043F0020332E0B3F5006F4DD017D8B3F5FA
:1021D000A06F31D0A3F5C063012B90D8636820466F
:1021E00094F882205E6894F88310B4F88430B04785
:1021F000002884D0436863670368A3671AE0B3F5D7
:10220000106F36D040F6024293427FF478AF5C4BB9
:1022100063670223A3670023C3E794F88230012B8E
:102220007FF46DAFB4F8883023F00203A4F888304F
:10223000C4E91D55E56778E7B4F88030B3F5A06FC1
:102240000ED194F88230204684F88A3001F034FAB6
:1022500063681B6813B1012120469847032323704C
:102260000023C4E91D339CE704F18B03636701235A
:10227000C3E72378042B10D1302383F31188204641
:10228000FFF7BAFE85F311880321636884F88B5049
:1022900021701B680BB12046984794F88230002BC0
:1022A000DED084F88B300423237063681B68002B16
:1022B000D6D0022120469847D2E794F884302046B1
:1022C0001D0603F00F010AD501F0A6FA012804D07B
:1022D00002287FF414AF2B4B9AE72B4B98E701F0C1
:1022E0008DFAF3E794F88230002B7FF408AF94F86E
:1022F000843013F00F01B3D01A06204602D501F046
:10230000AFFDADE701F0A0FDAAE794F88230002B05
:102310007FF4F5AE94F8843013F00F01A0D01B06C3
:10232000204602D501F084FD9AE701F075FD97E79C
:10233000142284F8702083F311882B462A462946FC
:102340002046FFF769FE85F31188E9E65DB11522A5
:1023500084F8702083F3118800212046D4E91D23DE
:10236000FFF75AFEFDE60B2284F8702083F31188F4
:102370002B462A4629462046FFF760FEE3E700BFCA
:10238000C4570008BC570008C057000838B590F87B
:1023900070300446002B3ED0063BDAB20F2A34D808
:1023A0000F2B32D8DFE803F03731310822323131D8
:1023B0003131313131313737856FB0F886309D4258
:1023C00014D2C3681B8AB5FBF3F203FB12556DB937
:1023D000302383F311882B462A462946FFF72EFE29
:1023E00085F311880A2384F870300EE0142384F8F2
:1023F0007030302383F31188002320461A46194693
:10240000FFF70AFE002383F3118838BDC36F03B1C1
:1024100098470023E7E70021204601F009FD00214D
:10242000204601F0F9FC63681B6813B106212046C1
:1024300098470623D7E7000010B590F8703004469F
:10244000142B29D017D8062B05D001D81BB110BDED
:10245000093B022BFBD80021204601F0E9FC0021BA
:10246000204601F0D9FC63681B6813B106212046A1
:102470009847062319E0152BE9D10B2380F870301B
:10248000302383F3118800231A461946FFF7D6FD3F
:10249000002383F31188DAE7C3689B695B68002B2C
:1024A000D5D1C36F03B19847002384F87030CEE7CD
:1024B00000238268037503691B6899689142FBD207
:1024C0005A68036042601060586070470023826859
:1024D000037503691B6899689142FBD85A680360C9
:1024E000426010605860704708B50846302383F397
:1024F00011880A7D0023052A06D8DFE802F00B05C3
:102500000503120E826913604FF0FF338361FFF7FA
:10251000CFFF002383F3118808BD826993680133DC
:102520009360D0E9003213605A60EDE7FFF7C0BF57
:1025300038B50A4B1C68DD682875226853601A603C
:102540000122DC60A3682275934201D100F060FE95
:1025500029462046BDE83840FDF754BFC828002072
:102560000C4B30B5DD684B1C87B004460FD02B46B2
:10257000094A684600F092F92046FFF7D9FF009B10
:1025800013B1684600F094F9A86907B030BDFFF7B1
:10259000CFFFF9E7C8280020E924000870B50F4EE6
:1025A00004468161F36881689A68914203D8BDE866
:1025B0007040FFF77DBF1846FFF788FF8368054628
:1025C000012B01D100F026FE012329462046F460AC
:1025D0002375BDE87040FDF715BF00BFC828002077
:1025E000044B1A68DB6890689B68984294BF00208F
:1025F00001207047C828002038B50B4B1C68DD68E7
:10260000226853601A600122DC602275AB68934235
:1026100001D100F0FFFD2846FFF758FF0146204694
:10262000BDE83840FDF7EEBEC828002038B50123CC
:10263000084C00252370656001F000FE01F026FEC5
:102640000549064801F0FAFE0223237085F311883C
:1026500038BD00BF302B0020CC570008C828002010
:1026600000F05CB9034A516853685B1A9842FBD882
:10267000704700BF001000E08B600223086108462D
:102680008B8270478368A3F1840243F8142C02699B
:1026900043F8442C426943F8402C094A43F8242C5F
:1026A000C268A3F1200043F8182C022203F80C2C76
:1026B000002203F80B2C034A43F8102C704700BF8C
:1026C0001D040008C828002008B5FFF7DBFFBDE89F
:1026D0000840FFF72BBF0000024BDB6898610F201A
:1026E000FFF726BFC8280020302383F31188FFF7A7
:1026F000F3BF000008B50146302383F3118808209A
:10270000FFF72EFF002383F3118808BD054BDB681C
:1027100021B1036098610320FFF722BF4FF0FF3023
:10272000704700BFC828002003682BB10022026058
:1027300018469961FFF7FABE70470000064BDB6848
:1027400039B1426818605A60136043600420FFF793
:1027500007BF4FF0FF307047C82800200368984239
:1027600006D01A680260506018469961FFF7DEBE15
:102770007047000038B504460D462068844200D1F9
:1027800038BD036823605C608561FFF7CFFEF4E726
:10279000036810B59C68A2420CD85C688A600B6024
:1027A0004C602160596099688A1A9A604FF0FF3333
:1027B000836010BD121B1B68ECE700000A2938BFBC
:1027C0000A2170B504460D460A26601901F032FD53
:1027D00001F01EFD041BA54203D8751C04462E46BD
:1027E000F3E70A2E04D90120BDE8704001F066BE6F
:1027F00070BD0000F8B5144B0D460A2A4FF00A07C9
:10280000D96103F11001826038BF0A224160196961
:102810001446016048601861A81801F0FDFC01F041
:10282000F7FC431B0646A34206D37C1C2819274607
:10283000354601F0FFFCF2E70A2F04D90120BDE87C
:10284000F84001F03BBEF8BDC8280020F8B50646A8
:102850000D4601F0DDFC0F4A134653F8107F9F42EE
:1028600006D12A4601463046BDE8F840FFF7C2BF10
:10287000D169BB68441A2C1928BF2C46A34202D93F
:102880002946FFF79BFF224631460348BDE8F84042
:10289000FFF77EBFC8280020D8280020C0E9032306
:1028A000002310B45DF8044B4361FFF7CFBF000075
:1028B00010B5194C236998420DD08168D0E90032D7
:1028C00013605A609A680A449A60002303604FF0CC
:1028D000FF33A36110BD0268234643F8102F5360F5
:1028E0000022026022699A4203D1BDE8104001F043
:1028F0009BBC936881680B44936001F089FC22695A
:10290000E1699268441AA242E4D91144BDE810403A
:10291000091AFFF753BF00BFC82800202DE9F04770
:10292000DFF8BC8008F110072C4ED8F8105001F0E9
:102930006FFCD8F81C40AA68031B9A423ED8144486
:102940004FF00009D5E90032C8F81C4013605A6006
:10295000C5F80090D8F81030B34201D101F064FC02
:1029600089F31188D5E9033128469847302383F34A
:1029700011886B69002BD8D001F04AFC6A69A0EB82
:10298000040982464A450DD2022001F097FD00223B
:10299000D8F81030B34208D151462846BDE8F04778
:1029A000FFF728BF121A2244F2E712EB0909294661
:1029B000384638BF4A46FFF7EBFEB5E7D8F8103087
:1029C000B34208D01444C8F81C00211AA960BDE81D
:1029D000F047FFF7F3BEBDE8F08700BFD82800201E
:1029E000C828002000207047FEE700007047000064
:1029F0004FF0FF307047000002290CD0032904D0AB
:102A00000129074818BF00207047032A05D8054848
:102A100000EBC2007047044870470020704700BFB9
:102A2000A4580008442200205858000870B59AB0F5
:102A300005460846144601A900F0C2F801A8FEF7B1
:102A400051FA431C0022C6B25B001046C5E90034AF
:102A500023700323023404F8013C01ABD1B20234E9
:102A60008E4201D81AB070BD13F8011B013204F870
:102A7000010C04F8021CF1E708B5302383F3118838
:102A80000348FFF7F7F9002383F3118808BD00BF5F
:102A9000382B002090F8803003F01F02012A07D164
:102AA00090F881200B2A03D10023C0E91D3315E0E3
:102AB00003F06003202B08D1B0F884302BB990F8D4
:102AC0008120212A03D81F2A04D8FFF7B5B9222A6A
:102AD000EBD0FAE7034A426707228267C367012007
:102AE000704700BF3B22002007B5052917D8DFE853
:102AF00001F0191603191920302383F31188104AA5
:102B000001210190FFF75EFA019802210D4AFFF7BB
:102B100059FA0D48FFF77AF9002383F3118803B0BF
:102B20005DF804FB302383F311880748FFF744F96D
:102B3000F2E7302383F311880348FFF75BF9EBE7F3
:102B4000F85700081C580008382B002038B50C4DE9
:102B50000C4C2A460C4904F10800FFF767FF05F109
:102B6000CA0204F110000949FFF760FF05F5CA72B7
:102B700004F118000649BDE83840FFF757BF00BF11
:102B80001044002044220020D8570008E2570008D3
:102B9000ED57000870B5044608460D46FEF7A2F949
:102BA000C6B22046013403780BB9184670BD3246D0
:102BB0002946FEF783F90028F3D10120F6E700004B
:102BC0002DE9F04705460C46FEF78CF92B49C6B2B5
:102BD0002846FFF7DFFF08B10636F6B22849284637
:102BE000FFF7D8FF08B11036F6B2632E0BD8DFF826
:102BF0008C80DFF88C90234FDFF894A02E7846B9B4
:102C00002670BDE8F08729462046BDE8F04702F06F
:102C1000EBBC252E2ED1072241462846FEF74EF961
:102C200070B9194B224603F10C0153F8040B8B4287
:102C300042F8040BF9D11B7807350D341370DDE72A
:102C4000082249462846FEF739F998B9A21C0F4BCD
:102C5000197802320909C95D02F8041C13F8011B36
:102C600001F00F015345C95D02F8031CF0D118347F
:102C70000835C3E7013504F8016BBFE7C458000805
:102C8000ED570008DA580008CC58000800E8F11F9A
:102C90000CE8F11FBFF34F8F044B1A695107FCD1A9
:102CA000D3F810215207F8D1704700BF002000521E
:102CB00008B50D4B1B78ABB9FFF7ECFF0B4BDA688F
:102CC000D10704D50A4A5A6002F188325A60D3F813
:102CD0000C21D20706D5064AC3F8042102F1883236
:102CE000C3F8042108BD00BF6E460020002000523A
:102CF0002301674508B5114B1B78F3B9104B1A69CE
:102D0000510703D5DA6842F04002DA60D3F81021A7
:102D1000520705D5D3F80C2142F04002C3F80C212C
:102D2000FFF7B8FF064BDA6842F00102DA60D3F829
:102D30000C2142F00102C3F80C2108BD6E460020B0
:102D4000002000520F289ABF00F580604004002048
:102D5000704700004FF400307047000010207047AB
:102D60000F2808B50BD8FFF7EDFF00F50033026818
:102D7000013204D104308342F9D1012008BD002082
:102D8000FCE700000F2838B505463FD8FFF782FF63
:102D90001F4CFFF78DFF4FF0FF3307286361C4F826
:102DA00014311DD82361FFF775FF030243F024039C
:102DB000E360E36843F08003E36023695A07FCD4CF
:102DC0002846FFF767FFFFF7BDFF4FF4003100F023
:102DD000E5F92846FFF78EFFBDE83840FFF7C0BF92
:102DE000C4F81031FFF756FFA0F108031B0243F0AF
:102DF0002403C4F80C31D4F80C3143F08003C4F838
:102E00000C31D4F810315B07FBD4D9E7002038BD72
:102E1000002000522DE9F84F04460D46104644EAC2
:102E20000203DE0602D00020BDE8F88F20F01F006C
:102E3000DFF8D4B0DFF8D4A0FFF73AFF05EB0008C5
:102E4000454503D10120FFF755FFEDE72022294634
:102E5000204602F0B9FB10B920342035F0E72346B4
:102E600004F120021F68791CDDD104339342F9D1AB
:102E700004F178432048214EB3F5801F204B38BF22
:102E8000184603F1F80332BFD946D1461E46FFF774
:102E900001FF0760A4EB050C336805F11C0143F04A
:102EA000020333602B1FD9F8007017F00507FAD121
:102EB00053F8042F8B424CF80320F4D1BFF34F8F0B
:102EC000FFF7E8FE4FF0FF330360336823F002039F
:102ED0003360BFF34F8F0B4BC3F85C42BFF34F8F90
:102EE000BFF36F8F20222946204602F06DFB002899
:102EF000B2D03846A7E700BF142100520C20005280
:102F00001420005200ED00E0102000521021005269
:102F100010B5084C237828B11BB9FFF7C9FE01236F
:102F2000237010BD002BFCD02070BDE81040FFF7CF
:102F3000E1BE00BF6E4600202DE9F04F0D4685B082
:102F4000814658B111F00D0614BF2022082211F05D
:102F50000803019304D0431E03426AD0002435E0E5
:102F6000002E37D009F11F0121F01F094FF0010891
:102F7000324F05F00403DFF8D0A005EA080BBBF1DF
:102F8000000F32D07869C0072FD408F101080C3740
:102F9000B8F1060FF3D19EB9294D4946A8190192FF
:102FA00001F096F9044600283AD11836019A782E95
:102FB000F3D1494601F08CF90446002830D1019A3A
:102FC0004946204801F084F9044668BB204605B014
:102FD000BDE8F08F0029C9D101462846029201F0D0
:102FE00077F90446E0B9029AC0E713B1786941075E
:102FF000CBD5AC0702D578698007C6D5019911B148
:1030000078690107C1D51820494600FB08A0CDE921
:10301000022301F05DF90446DDE902230028B4D063
:103020004A460021204601E04A460021FDF762FFA2
:10303000CCE70246002E95D198E700BFEC58000877
:10304000A046002070460020884600200121FFF79E
:1030500073BF0000F8B500231A461A600433B3F5B5
:10306000806FFAD1114D01241827114E07FB04601F
:1030700001342A6955F80C1F01F016F9062CF5D118
:1030800037254FF4C0542046FFF7E0FF014628B132
:1030900022460848BDE8F84001F006B9C4EBC40474
:1030A000013D4FEAD404EED1F8BD00BFEC58000852
:1030B00088460020704600200421FFF73DBF000035
:1030C00008B101F077B9704770B5AAB140EA0103C1
:1030D00013F01F030FD1094C0144A5686D0706D5F5
:1030E0002568A84203D366683544A94204D903334E
:1030F0000C34122BF1D10022104670BDEC580008A0
:103100000244074BD2B210B5904200D110BD441C0E
:1031100000B253F8200041F8040BE0B2F4E700BF1E
:10312000504000580E4B30B51C6F240405D41C6F62
:103130001C671C6F44F400441C670A4C024423685B
:10314000D2B243F480732360074B904200D130BD6C
:10315000441C51F8045B00B243F82050E0B2F4E79D
:1031600000440258004802585040005807B5012258
:1031700001A90020FFF7C4FF019803B05DF804FB2C
:1031800013B50446FFF7F2FFA04205D0012201A9C2
:1031900000200194FFF7C6FF02B010BD0144BFF349
:1031A0004F8F064B884204D3BFF34F8FBFF36F8F0F
:1031B0007047C3F85C022030F4E700BF00ED00E088
:1031C0000144BFF34F8F064B884204D3BFF34F8FA8
:1031D000BFF36F8F7047C3F870022030F4E700BF71
:1031E00000ED00E0034B1A681AB9034AD2F8D02464
:1031F0001A607047184700200040025808B5FFF7D2
:10320000F1FF024B1868C0F3806008BD184700202A
:103210007047000070470000EFF3098305496833E9
:103220004A6B22F001024A6383F30988002383F387
:103230001188704700EF00E0302080F3118862B6FB
:103240000D4B0E4AD96821F4E0610904090C0A43C8
:103250000B49DA60D3F8FC2042F08072C3F8FC20FE
:10326000084AC2F8B01F116841F001011160202224
:10327000DA7783F82200704700ED00E00003FA05DA
:1032800055CEACC5001000E0302310B583F3118893
:103290000E4B5B6813F4006314D0F1EE103AEFF3B9
:1032A00009844FF08073683CE361094BDB6B236654
:1032B00084F30988FFF794F910B1064BA36110BDA0
:1032C000054BFBE783F31188F9E700BF00ED00E051
:1032D00000EF00E02F0400083204000870B5BFF3CF
:1032E0004F8FBFF36F8F1A4A0021C2F85012BFF3FD
:1032F0004F8FBFF36F8F536943F400335361BFF3B4
:103300004F8FBFF36F8FC2F88410BFF34F8FD2F887
:10331000803043F6E074C3F3C900C3F34E335B015E
:1033200003EA0406014646EA81750139C2F8605293
:10333000F9D2203B13F1200FF2D1BFF34F8F536925
:1033400043F480335361BFF34F8FBFF36F8F70BD72
:1033500000ED00E0FEE70000214B2248224A70B554
:10336000904237D3214BC11EDA1C121A22F00302FD
:103370008B4238BF00220021FDF7BCFD1C4A002310
:10338000C2F88430BFF34F8FD2F8803043F6E07438
:10339000C3F3C900C3F34E335B0103EA04060146DD
:1033A00046EA81750139C2F86C52F9D2203B13F11B
:1033B000200FF2D1BFF34F8FBFF36F8FBFF34F8F4B
:1033C000BFF36F8F0023C2F85032BFF34F8FBFF3AC
:1033D0006F8F70BD53F8041B40F8041BC0E700BF9B
:1033E0003C5B0008E44A0020E44A0020E44A002054
:1033F00000ED00E0074BD3F8D81021EA0001C3F834
:10340000D810D3F8002122EA0002C3F80021D3F833
:10341000003170470044025870B5D0E924430022BF
:103420004FF0FF359E6804EB42135101D3F80009B9
:10343000002805DAD3F8000940F08040C3F80009FD
:10344000D3F8000B002805DAD3F8000B40F08040D9
:10345000C3F8000B013263189642C3F80859C3F849
:10346000085BE0D24FF00113C4F81C3870BD0000B7
:10347000890141F02001016103699B06FCD41220FF
:10348000FFF7F0B810B50A4C2046FEF779FD094B5E
:10349000C4F89030084BC4F89430084C2046FEF72E
:1034A0006FFD074BC4F89030064BC4F8943010BD44
:1034B0001C4700200000084058590008B847002069
:1034C000000004406459000870B503780546012BDC
:1034D0005CD1434BD0F89040984258D1414B0E21DB
:1034E0006520D3F8D82042F00062C3F8D820D3F882
:1034F000002142F00062C3F80021D3F80021D3F884
:10350000802042F00062C3F88020D3F8802022F0AF
:103510000062C3F88020D3F88030FEF797F9324B71
:10352000E360324BC4F800380023D5F89060C4F84B
:10353000003EC02323604FF40413A3633369002BC0
:10354000FCDA01230C203361FFF78CF83369DB07C9
:10355000FCD41220FFF786F83369002BFCDA002632
:103560002846A660FFF758FF6B68C4F81068DB6850
:10357000C4F81468C4F81C6883BB1D4BA3614FF0EA
:10358000FF336361A36843F00103A36070BD194B6F
:103590009842C9D1134B4FF08060D3F8D82042F045
:1035A0000072C3F8D820D3F8002142F00072C3F8AB
:1035B0000021D3F80021D3F8802042F00072C3F834
:1035C0008020D3F8802022F00072C3F88020D3F846
:1035D0008030FFF70FFF0E214D209EE7064BCDE711
:1035E0001C47002000440258401400400300200201
:1035F000003C30C0B8470020083C30C0F8B5D0F8D7
:103600009040054600214FF000662046FFF730FF4E
:10361000D5F8941000234FF001128F684FF0FF305F
:10362000C4F83438C4F81C2804EB431201339F4219
:10363000C2F80069C2F8006BC2F80809C2F8080BAA
:10364000F2D20B68D5F89020C5F898306362102349
:103650001361166916F01006FBD11220FFF702F86D
:10366000D4F8003823F4FE63C4F80038A36943F4A7
:10367000402343F01003A3610923C4F81038C4F8B1
:1036800014380B4BEB604FF0C043C4F8103B094BB0
:10369000C4F8003BC4F81069C4F80039D5F8983074
:1036A00003F1100243F48013C5F89820A362F8BD1B
:1036B0003459000840800010D0F8902090F88A100B
:1036C000D2F8003823F4FE6343EA0113C2F800384D
:1036D000704700002DE9F84300EB8103D0F89050CB
:1036E0000C468046DA680FFA81F94801166806F040
:1036F0000306731E022B05EB41134FF0000194BF2C
:10370000B604384EC3F8101B4FF0010104F110034A
:1037100098BF06F1805601FA03F3916998BF06F548
:10372000004600293AD0578A04F15801374349012D
:103730006F50D5F81C180B430021C5F81C382B1806
:103740000127C3F81019A7405369611E9BB3138A60
:10375000928B9B08012A88BF5343D8F89820981869
:1037600042EA034301F140022146C8F89800284686
:1037700005EB82025360FFF77BFE08EB8900C3680C
:103780001B8A43EA845348341E4364012E51D5F802
:103790001C381F43C5F81C78BDE8F88305EB4917B2
:1037A000D7F8001B21F40041C7F8001BD5F81C18FE
:1037B00021EA0303C0E704F13F030B4A28462146F0
:1037C00005EB83035A60FFF753FE05EB4910D0F871
:1037D000003923F40043C0F80039D5F81C3823EA37
:1037E0000707D7E70080001000040002D0F89420FB
:1037F0001268C0F89820FFF70FBE00005831D0F8CB
:10380000903049015B5813F4004004D013F4001FBA
:103810000CBF0220012070474831D0F89030490198
:103820005B5813F4004004D013F4001F0CBF0220B7
:103830000120704700EB8101CB68196A0B681360A7
:103840004B6853607047000000EB810330B5DD68C2
:10385000AA691368D36019B9402B84BF4023136051
:103860006B8A1468D0F890201C4402EB4110013C94
:1038700009B2B4FBF3F46343033323F0030343EAD5
:10388000C44343F0C043C0F8103B2B6803F003036C
:10389000012B0ED1D2F8083802EB411013F4807FCF
:1038A000D0F8003B14BF43F0805343F00053C0F8FE
:1038B000003B02EB4112D2F8003B43F00443C2F854
:1038C000003B30BD2DE9F041D0F8906005460C4634
:1038D00006EB4113D3F8087B3A07C3F8087B08D5F9
:1038E000D6F814381B0704D500EB8103DB685B684E
:1038F0009847FA071FD5D6F81438DB071BD505EB18
:103900008403D968CCB98B69488A5A68B2FBF0F64F
:1039100000FB16228AB91868DA6890420DD2121A92
:10392000C3E90024302383F3118821462846FFF79A
:103930008BFF84F31188BDE8F081012303FA04F2C0
:103940006B8923EA02036B81CB68002BF3D02146FD
:103950002846BDE8F041184700EB81034A0170B5E5
:10396000DD68D0F890306C692668E66056BB1A4472
:103970004FF40020C2F810092A6802F00302012A5D
:103980000AB20ED1D3F8080803EB421410F4807F7A
:10399000D4F8000914BF40F0805040F00050C4F843
:1039A000000903EB4212D2F8000940F00440C2F8CB
:1039B00000090122D3F8340802FA01F10143C3F8E7
:1039C000341870BD19B9402E84BF40202060206893
:1039D0001A442E8A8419013CB4FBF6F440EAC44030
:1039E00040F00050C6E700002DE9F843D0F89060A1
:1039F00005460C464F0106EB4113D3F8088918F031
:103A0000010FC3F808891CD0D6F81038DB0718D589
:103A100000EB8103D3F80CC0DCF81430D3F800E0DD
:103A2000DA68964530D2A2EB0E024FF000091A6018
:103A3000C3F80490302383F31188FFF78DFF89F3D7
:103A4000118818F0800F1DD0D6F834380126A64012
:103A5000334217D005EB84030134D5F89050D3F8E6
:103A60000CC0E4B22F44DCF8142005EB0434D2F887
:103A700000E05168714514D3D5F8343823EA0606BE
:103A8000C5F83468BDE8F883012303FA01F203891D
:103A900023EA02030381DCF80830002BD1D09847D9
:103AA000CFE7AEEB0103BCF81000834228BF03460A
:103AB000D7F8180980B2B3EB800FE3D89068A0F173
:103AC000040959F8048FC4F80080A0EB0908984451
:103AD000B8F1040FF5D818440B4490605360C8E760
:103AE0002DE9F84FD0F8905004466E69AB691E403E
:103AF00016F480586E6103D0BDE8F84FFEF7B0BAF7
:103B0000002E12DAD5F8003E9B0705D0D5F8003E0E
:103B100023F00303C5F8003ED5F80438204623F00F
:103B20000103C5F80438FEF7C9FA370505D5204664
:103B3000FFF772FC2046FEF7AFFAB0040CD5D5F8BB
:103B4000083813F0060FEB6823F470530CBF43F4EE
:103B5000105343F4A053EB6031071BD56368DB6857
:103B60001BB9AB6923F00803AB612378052B0CD19B
:103B7000D5F8003E9A0705D0D5F8003E23F00303A0
:103B8000C5F8003E2046FEF799FA6368DB680BB182
:103B900020469847F30200F1BA80B70226D5D4F840
:103BA000909000274FF0010A09EB4712D2F8003B32
:103BB00003F44023B3F5802F11D1D2F8003B002B42
:103BC0000DDA62890AFA07F322EA0303638104EB40
:103BD0008703DB68DB6813B1394620469847013715
:103BE000D4F89430FFB29B689F42DDD9F00619D516
:103BF000D4F89000026AC2F30A1702F00F0302F42D
:103C0000F012B2F5802F00F0CA80B2F5402F09D132
:103C100004EB8303002200F58050DB681B6A9742A7
:103C200040F0B0803003D5F8185835D5E90303D5F6
:103C300000212046FFF746FEAA0303D501212046B6
:103C4000FFF740FE6B0303D502212046FFF73AFE43
:103C50002F0303D503212046FFF734FEE80203D5E6
:103C600004212046FFF72EFEA90203D50521204698
:103C7000FFF728FE6A0203D506212046FFF722FE41
:103C80002B0203D507212046FFF71CFEEF0103D5C9
:103C900008212046FFF716FE700340F1A780E907D0
:103CA00003D500212046FFF79FFEAA0703D5012177
:103CB0002046FFF799FE6B0703D502212046FFF748
:103CC00093FE2F0703D503212046FFF78DFEEE0656
:103CD00003D504212046FFF787FEA80603D505215A
:103CE0002046FFF781FE690603D506212046FFF72F
:103CF0007BFE2A0603D507212046FFF775FEEB055C
:103D000074D520460821BDE8F84FFFF76DBED4F802
:103D100090904FF0000B4FF0010AD4F894305FFA06
:103D20008BF79B689F423FF638AF09EB4713D3F8F8
:103D3000002902F44022B2F5802F20D1D3F80029C7
:103D4000002A1CDAD3F8002942F09042C3F8002977
:103D5000D3F80029002AFBDB3946D4F89000FFF79E
:103D600087FB22890AFA07F322EA0303238104EB83
:103D70008703DB689B6813B13946204698470BF1EF
:103D8000010BCAE7910701D1D0F80080072A02F1A0
:103D900001029CBF03F8018B4FEA18283FE704EBB0
:103DA000830300F58050DA68D2F818C0DCF80820E8
:103DB000DCE9001CA1EB0C0C00218F4208D1DB6870
:103DC0009B699A683A449A605A683A445A6029E76B
:103DD00011F0030F01D1D0F800808C4501F10101F1
:103DE00084BF02F8018B4FEA1828E6E7BDE8F88F98
:103DF00008B50348FFF774FEBDE80840FFF744BA72
:103E00001C47002008B50348FFF76AFEBDE80840DC
:103E1000FFF73ABAB8470020D0F8903003EB4111D1
:103E2000D1F8003B43F40013C1F8003B7047000099
:103E3000D0F8903003EB4111D1F8003943F400136E
:103E4000C1F8003970470000D0F8903003EB411101
:103E5000D1F8003B23F40013C1F8003B7047000089
:103E6000D0F8903003EB4111D1F8003923F400135E
:103E7000C1F800397047000030B50433039C01726B
:103E8000002104FB0325C160C0E90653049B0363C2
:103E9000059BC0E90000C0E90422C0E90842C0E96E
:103EA0000A11436330BD00000022416AC260C0E9CC
:103EB0000411C0E90A226FF00101FEF75BBC0000AB
:103EC000D0E90432934201D1C2680AB9181D704783
:103ED00000207047036919600021C2680132C26086
:103EE000C269134482699342036124BF436A036138
:103EF000FEF734BC38B504460D46E3683BB1626951
:103F00000020131D1268A3621344E36207E0237AC2
:103F100033B929462046FEF711FC0028EDDA38BDFA
:103F20006FF00100FBE70000C368C269013BC3609A
:103F30004369134482699342436124BF436A4361E6
:103F400000238362036B03B11847704770B53023B9
:103F5000044683F31188866A3EB9FFF7CBFF054616
:103F600018B186F31188284670BDA36AE26A13F877
:103F7000015B9342A36202D32046FFF7D5FF0023E3
:103F800083F31188EFE700002DE9F84F04460E4651
:103F9000174698464FF0300989F311880025AA4644
:103FA000D4F828B0BBF1000F09D141462046FFF7F5
:103FB000A1FF20B18BF311882846BDE8F88FD4E922
:103FC0000A12A7EB050B521A934528BF9346BBF183
:103FD000400F1BD9334601F1400251F8040B9142C6
:103FE00043F8040BF9D1A36A403640354033A3624D
:103FF000D4E90A239A4202D32046FFF795FF8AF3B9
:104000001188BD42D8D289F31188C9E730465A4693
:10401000FCF74AFFA36A5E445D445B44A362E7E7A2
:1040200010B5029C0433017203FB0421C460C0E993
:1040300006130023C0E90A33039B0363049BC0E912
:104040000000C0E90422C0E90842436310BD00003B
:10405000026A6FF00101C260426AC0E904220022D4
:10406000C0E90A22FEF786BBD0E904239A4201D1B7
:10407000C26822B9184650F8043B0B607047002311
:104080001846FAE7C3680021C2690133C360436977
:10409000134482699342436124BF436A4361FEF73C
:1040A0005DBB000038B504460D46E3683BB12369AB
:1040B00000201A1DA262E2691344E36207E0237A3A
:1040C00033B929462046FEF739FB0028EDDA38BD22
:1040D0006FF00100FBE7000003691960C268013A54
:1040E000C260C269134482699342036124BF436A78
:1040F000036100238362036B03B11847704700001C
:1041000070B530230D460446114683F31188866A44
:104110002EB9FFF7C7FF10B186F3118870BDA36AEF
:104120001D70A36AE26A01339342A36204D3E1697A
:1041300020460439FFF7D0FF002080F31188EDE717
:104140002DE9F84F04460D46904699464FF0300A47
:104150008AF311880026B346A76A4FB9494620461C
:10416000FFF7A0FF20B187F311883046BDE8F88F34
:10417000D4E90A073A1AA8EB0607974228BF174660
:10418000402F1BD905F1400355F8042B9D4240F800
:10419000042BF9D1A36A40364033A362D4E90A2341
:1041A0009A4204D3E16920460439FFF795FF8BF367
:1041B00011884645D9D28AF31188CDE729463A4677
:1041C000FCF772FEA36A3D443E443B44A362E5E72C
:1041D000D0E904239A4217D1C3689BB1836A8BB19B
:1041E000043B9B1A0ED01360C368013BC360C369D4
:1041F0001A4483699A42026124BF436A036100231F
:1042000083620123184670470023FBE700F05EBA83
:104210004FF08043586A70474FF080430022586344
:104220001A610222DA6070474FF080430022DA60A0
:10423000704700004FF0804358637047024B034AB9
:104240001A60034A5A6070476C480020E84A002010
:1042500000000220074B494210B55C68201A084054
:104260001968821A8A4203D3A24201D85A6010BD4B
:104270000020FCE76C48002008B5302383F3118848
:10428000FFF7E8FF002383F3118808BD04480121EC
:10429000044B03600023C0E901330C3000F016B971
:1042A0007448002079420008CB1D083A23F0070328
:1042B000591A521A012110B4D2080024C0E900434F
:1042C00084600C301C605A605DF8044B00F0FEB84E
:1042D0002DE9F84F364ECD1D0F46002818BF064673
:1042E000082A4FEAD50538BF082206F10C08341D0C
:1042F0009146404600F006F909F10701C9F1000EA8
:10430000224624686CB9404600F006F93368CBB306
:1043100008224946E8009847044698B340E90267F6
:1043200030E004EB010CD4F804A00CEA0E0C0AF106
:104330000100ACF1080304EBC0009842E0D9A0EB07
:104340000C0CB5EBEC0F4FEAEC0BD9D89C421CD20D
:1043500004F10802AB45A3EB02024FEAE2026260FD
:1043600009D9691CED43206803EBC1025D44556027
:1043700043F8310022601C465F60404644F8086BF9
:1043800000F0CAF82046BDE8F88FAA45216802D19E
:1043900011602346EFE7013504EBC50344F83510FF
:1043A00003F10801401AC01058601360F1E700BF24
:1043B00074480020F8B550F8043C044650F8085CF6
:1043C000A0F1080607332F1D0C35DB0840F8043C2C
:1043D000284600F097F83B469F421A6801D0B34246
:1043E00028D20AB1964225D244F8082C54F8042C5D
:1043F0001E60013254F8081C06EBC200814206D14F
:104400004868024444F8042C0A6844F8082C5868A8
:10441000411C03EBC1018E4207D154F8042C013238
:1044200002445A6054F8082C1A602846BDE8F84047
:1044300000F072B81346CFE7FEE7000070B51B4BE3
:104440000025044686B058600E4685620163FEF77B
:10445000F3FE04F11003A560E562C4E904334FF0F4
:10446000FF33C4E90044C4E90635FFF7D1FE2B460B
:10447000024604F134012046C4E9082380230C4A93
:104480002565FEF7F9F801230A4AE06000920375FA
:10449000684672680192B268CDE90223064BCDE905
:1044A0000435FEF711F906B070BD00BF302B0020B7
:1044B000705900087559000839440008024AD36A47
:1044C0001843D062704700BFC8280020C0E9000030
:1044D000816070478368013B002B10B583600CDA64
:1044E000074BDC684368A061206063601C60446027
:1044F0000520FEF71DF8A06910BD0020FCE700BFF5
:10450000C828002008B5302383F31188FFF7E2FFA5
:10451000002383F3118808BD08B5302383F3118885
:1045200083680133002B836007DC036800211A686D
:10453000026050601846FEF731F8002383F31188BB
:1045400008BD00004B6843608B688360CB68C36024
:104550000B6943614B6903628B6943620B680360BB
:104560007047000008B53C4B40F2FF713B48D3F860
:1045700088200A43C3F88820D3F8882022F4FF62F9
:1045800022F00702C3F88820D3F88820D3F8E0206F
:104590000A43C3F8E020D3F808210A43C3F80821EE
:1045A0002F4AD3F808311146FFF7CCFF00F58060A1
:1045B00002F11C01FFF7C6FF00F5806002F138012F
:1045C000FFF7C0FF00F5806002F15401FFF7BAFF6A
:1045D00000F5806002F17001FFF7B4FF00F5806024
:1045E00002F18C01FFF7AEFF00F5806002F1A80137
:1045F000FFF7A8FF00F5806002F1C401FFF7A2FFFA
:1046000000F5806002F1E001FFF79CFF00F580609B
:1046100002F1FC01FFF796FF02F58C7100F5806056
:10462000FFF790FF00F01CF90E4BD3F8902242F0F8
:104630000102C3F89022D3F8942242F00102C3F899
:1046400094220522C3F898204FF06052C3F89C20B2
:10465000054AC3F8A02008BD0044025800000258D3
:104660007C59000800ED00E01F00080308B500F0C9
:10467000F1F9FDF7DBFF104BD3F8DC2042F04002EC
:10468000C3F8DC20D3F8042122F04002C3F804214F
:10469000D3F80431094B1A6842F008021A601A680C
:1046A00042F004021A60FEF79DFDFEF7D3FCBDE860
:1046B0000840FEF74BBA00BF0044025800180248F9
:1046C000012070470020704770470000114BD3F85D
:1046D000E82042F00102C3F8E820D3F8102142F0AC
:1046E0000102C3F810210C4AD3F81031D36B43F008
:1046F0000103D3634FF08043C7229A624FF0FF3229
:10470000DA6200229A615A63DA605A6001225A61C1
:104710001A607047004402580010005C4FF080425D
:1047200008B51169D3680B40D9B29B076FEA010144
:10473000116107D5302383F31188FDF791FF002322
:1047400083F3118808BD0000064BD3F8DC20024338
:10475000C3F8DC20D3F804211043C3F80401D3F8D4
:10476000043170470044025808B53C4B4FF0FF310C
:10477000D3F8802062F00042C3F88020D3F8802074
:1047800002F00042C3F88020D3F88020D3F88420C0
:10479000C3F88410D3F884200022C3F88420D3F80F
:1047A0008400D86F40F0FF4040F4FF0040F4DF4049
:1047B00040F07F00D867D86F20F0FF4020F4FF0062
:1047C00020F4DF4020F07F00D867D86FD3F888004E
:1047D0006FEA40506FEA5050C3F88800D3F8880061
:1047E000C0F30A00C3F88800D3F88800D3F890001B
:1047F000C3F89010D3F89000C3F89020D3F890003D
:10480000D3F89400C3F89410D3F89400C3F894201C
:10481000D3F89400D3F89800C3F89810D3F8980010
:10482000C3F89820D3F89800D3F88C00C3F88C1004
:10483000D3F88C00C3F88C20D3F88C00D3F89C00FC
:10484000C3F89C10D3F89C10C3F89C20D3F89C307C
:10485000FCF70EFEBDE8084000F0E8B8004402583E
:1048600008B50122534BC3F80821534BD3F8F42069
:1048700042F00202C3F8F420D3F81C2142F00202F5
:10488000C3F81C210222D3F81C314C4BDA605A6861
:104890009104FCD54A4A1A6001229A60494ADA60BA
:1048A00000221A614FF440429A61444B9A69920483
:1048B000FCD51A6842F480721A603F4B1A6F12F4EA
:1048C000407F04D04FF480321A6700221A671A68BA
:1048D00042F001021A60384B1A685007FCD50022DA
:1048E0001A611A6912F03802FBD1012119604FF0E8
:1048F000804159605A67344ADA62344A1A611A6848
:1049000042F480321A602C4B1A689103FCD51A6865
:1049100042F480521A601A689204FCD52C4A2D4940
:104920009A6200225A63196301F57C01DA6301F28D
:10493000E71199635A64284A1A64284ADA621A68A5
:1049400042F0A8521A601C4B1A6802F02852B2F1C9
:10495000285FF9D148229A614FF48862DA614022D7
:104960001A621F4ADA641F4A1A651F4A5A651F4AAB
:104970009A6532231E4A1360136803F00F03022B5B
:10498000FAD10D4A136943F003031361136903F06D
:104990003803182BFAD14FF00050FFF7D5FE4FF037
:1049A0008040FFF7D1FE4FF00040BDE80840FFF720
:1049B000CBBE00BF0080005100440258004802589E
:1049C00000C000F0020000010000FF010088900814
:1049D0002220400063020901470E0508DD0BBF01DC
:1049E00020000020000001100910E000000101106B
:1049F0000020005208B5034800F0E6FCBDE808407E
:104A0000FEF742BC8C48002008B50348FCF798FE2E
:104A1000BDE80840FEF738BC5C24002008B5FFF76D
:104A20007DFEBDE80840FEF72FBC000008B5092157
:104A30007A20FCF70BFF09213120FCF707FF072143
:104A40001C20FCF703FF0C215220BDE80840FCF7B6
:104A5000FDBE000008B5FFF787FE00F015FAFDF770
:104A6000B3F800F003FAFDF789FAFDF75BF9FFF7F9
:104A70002BFEBDE80840FFF7C9BB00000379052BFA
:104A800005BF836A002001204B6004BF4FF4007310
:104A90000B60704770B55D1E866A04460D44B542D2
:104AA00005D9436B43F080034363012070BD0625A5
:104AB000057100F03BFC05232371F7E770B55D1E1F
:104AC000866A04460D44B54205D9436B43F0800322
:104AD0004363012070BD0725057100F04DFC0523DF
:104AE0002371F7E738B505790446052D05D108236C
:104AF000037100F067FC257138BD0120FCE7000060
:104B00000323F0B5037185B0044600F001FA0022DA
:104B10002046114600F046FA4FF4D57203AB082147
:104B2000204600F061FA0246B8B901232363039BD3
:104B3000C3F30323012B09D103AB3721204600F037
:104B400053FA18B9A44B039A1340ABB12046012580
:104B500000F010FA0223237137E103AB0022372162
:104B6000204600F041FA28B99B4A039B1A40002ACC
:104B700000F0A78002232363236B03F00F03022BB3
:104B800040F0A9806425954E42F21070FDF7B2FD09
:104B900003AB32460121204600F010FA0028D5D19F
:104BA000039B002B80F293805A0003D5236B43F0C4
:104BB00010032363002204F108030221204600F0C1
:104BC00071FA02460028C1D104F1380303212046BE
:104BD00000F00AFA0028B9D104F11805A26B0921E6
:104BE00020462B4600F05EFA0028AFD102ABA26B44
:104BF0000721204600F0F8F906460028A6D1236BCD
:104C000003F00F03022B40F08F807E227F21284685
:104C100000F0E8FB012840F28780E76B42F2107059
:104C2000FDF768FD08234FF40072394620460096D0
:104C300000F054FA002889D1384600F021FC236B9B
:104C4000A06203F00F03022B72D103AB644A06216A
:104C5000204600F0C9F9002871D15F49039B194033
:104C6000B1FA81F14909204600F064F902AB4FF432
:104C700000721021204600F0B7F9054600287FF4A5
:104C800065AF554E029B33427FF460AF236B13F048
:104C90000E0F03F00F0273D0022A7FF457AFE36ABE
:104CA0001978012900F09480022900F093800029EE
:104CB00000F089804B4F204600F062F903AB3A4682
:104CC00076E011462046226300F06CF954E7013D7E
:104CD0007FF45AAF3AE7444D6426444A3E4F012BD5
:104CE00018BF154603AB00223721204600F07CF99F
:104CF00000287FF42BAF039B3B427FF427AF03AB2D
:104D00002A462921204600F059F900287FF41EAFD9
:104D1000039B002BFFF648AF013E3FF417AF42F272
:104D20001070FDF7E7FCDDE7284600F07DFB86E725
:104D30007E227F212846E66B00F054FB08B9002153
:104D400091E700234022314620460093062300F0DD
:104D5000C5F90028F3D1B3895BBA9B07EFD5244B83
:104D60004022314620460093062300F0B7F9002880
:104D7000E5D1317C01F00F010F3918BF012172E735
:104D8000E36A1978F9B101297FF4E0AE204600F01A
:104D9000F7F803ABA26B3721204600F025F9002875
:104DA0007FF4D4AE039B33427FF4D0AE03AB022238
:104DB0000621204600F018F900287FF4C7AE039BB7
:104DC00033427FF4C3AE05232371284605B0F0BDFE
:104DD000084F70E7084F6EE708E0FFFD0080FFC056
:104DE0000001B9030000B7030080FF5000001080ED
:104DF000F1FFFF800001B7030002B70337B5044697
:104E00000C4D01ABA26B0D21204600F0EDF878B9F6
:104E1000019B2B420BD1C3F34323042B08D0053B4A
:104E2000022B04D84FF47A70FDF764FCE9E7012007
:104E300003B030BD08E0FFFD70B53023054683F3B5
:104E4000118803790024022B03D184F311882046B2
:104E500070BD0423037184F311880226FFF7CEFF8F
:104E60000446284600F086F82E71F0E700F036B8C8
:104E7000044B03600123037100234363C0E90A3339
:104E8000704700BFB05A000870470000836CC26AC8
:104E90008B42506810B506D95A1E4C0002EB4103F4
:104EA000B3FBF4F3184410BD01F001038A0748BFB7
:104EB00043F002034A0748BF43F008030A0748BF0C
:104EC00043F00403CA0648BF43F010038A06426B4E
:104ED00048BF43F0200313434363704710B5074CAA
:104EE0002046FFF7C5FF064B0022C4E91023054BFF
:104EF000A364054BE363054BE36410BD8C480020BD
:104F00000070005200B4C404E0480020E04A0020D1
:104F100010B5446C0649FFF7B9FF6060236842F2A0
:104F2000107043F003032360BDE81040FDF7E2BBBF
:104F3000801A06000129F8B5466C0B4F09D1756837
:104F40000A493D40FFF7A2FF054345F480557560CF
:104F5000F8BD746806493C40FFF798FF044344F4E9
:104F600080547460F4E700BF00ECFFFF80F0FA02A9
:104F700040787D01436C00225A601A60704700003F
:104F8000426C0129536823F4404304D0022905D020
:104F900001B95360704743F48043FAE743F4004398
:104FA000F7E70000436C41F480519A60D9605A6B76
:104FB0001206FCD580229A637047000010B541F4B8
:104FC0008851446CA260E160616B11F04502FBD036
:104FD000A26311F0040203D0FFF766FF012010BDA9
:104FE000616910461960FAE710B541F48851446CC4
:104FF000A260E160616B11F04502FBD0A26311F089
:10500000050203D0FFF750FF012010BD6169104673
:105010001960FAE773B5134604460E46302282F350
:105020001188426CD26B32B14FF0FF3140300193A6
:10503000FDF76CFB019B606C00220265C263C262DB
:10504000456B15F4807504D185F31188012002B0F9
:1050500070BD4FF0FF31816382F31188012E06D9B4
:105060000C21204602B0BDE87040FFF7BDBF1046DE
:10507000EDE7000073B5446C0E4600250192616BAC
:10508000A1632565E562FFF70FFF012E07D9019B9C
:105090002A460C2102B0BDE87040FFF7A5BF02B060
:1050A00070BD000010B541F49851446CA260E160FD
:1050B000616B11F04502FBD0A26311F03F0203D0F7
:1050C000FFF7F2FE012010BD216A10461960E16968
:1050D0005960A16999606169D960F4E72DE9F743E6
:1050E00004460191006D01A91746984600F0D8F9D1
:1050F000064600284AD0626C2046DDF804905568C8
:10510000C5F3090501356B00A56CB5FBF3F54FF44C
:105110007A73B5FBF3F55D435562FFF76FFE50BB45
:10512000636C4FF0FF3201254146C3F8589020468A
:105130001D659A634FF49572DA6342F207029F622B
:10514000DA62E36C0A9AFFF74FFFA0B9E26C104BEA
:1051500011680B407BB929462046FFF75BFF0546E7
:1051600048B92E463A460199206D00F0D1F93046F3
:1051700003B0BDE8F0833A460199206D00F0C8F90C
:10518000E26C01212046FFF775FFF0E70126EEE70C
:1051900008E0FFFD2DE9F7431F46436C01924FF4F1
:1051A0007A725D6804468846C5F3090501356E00CC
:1051B000856CB5FBF6F5B5FBF2F555435D62FFF77F
:1051C0001DFE20B10125284603B0BDE8F0837E0214
:1051D00001A9206D324600F063F905460028F1D0A0
:1051E000636C019AD4F84C909A6501221A654FF0CD
:1051F000FF329A634FF49572DA639E62236BDB068B
:105200004B4658BF4FEA4828012F42461BD912216E
:105210002046FFF7E9FEC0B9D9F80020104B134033
:105220009BB9636C42F2930239462046DA62E26C23
:10523000FFF7F0FE804640B932460199206D4546A1
:1052400000F066F9BFE71121E2E732460199206DCF
:1052500000F05EF9E26C39462046FFF70BFFB2E73B
:1052600008E0FFFD2DE9F3411F46436C01924FF426
:105270007A725D6804468846C5F3090501356E00FB
:10528000856CB5FBF6F5B5FBF2F555435D62FFF7AE
:10529000B5FD20B10125284602B0BDE8F0817E02AF
:1052A00001A9206D324600F04BF905460028F1D0E7
:1052B000636C019A9A6501221A654FF0FF329A6376
:1052C0004FF48D72DA639E62236BE66CDB06334625
:1052D00058BF4FEA4828012F424619D919212046C4
:1052E000FFF782FEB0B932680F4B134093B9636C7D
:1052F00042F2910239462046DA62E26CFFF78AFEFA
:10530000064638B901993546206D00F055F9C2E7D7
:105310001821E4E70199206D00F04EF9E26C39465E
:105320002046FFF7A7FEB6E708E0FFFD12F0030FE7
:105330002DE9F04107460C4615461E4617D00E448F
:10534000B44202D10020BDE8F0810123FA6B21466E
:105350003846FFF71FFF0028F5D128464FF40072AA
:10536000F96B05F500750134FBF79EFDE8E7BDE834
:10537000F041FFF70FBF000012F0030F2DE9F041DD
:1053800007460C4615461E4617D00E44B44202D1BD
:105390000020BDE8F08129464FF40072F86B05F556
:1053A0000075FBF781FD0123FA6B21463846FFF7B4
:1053B00059FF0028EDD10134E8E7BDE8F041FFF7DF
:1053C00051BF000000207047302310B583F31188CF
:1053D0000024436C40302146DC63FDF7A5F984F3DB
:1053E000118810BD01F01F03F0B502F01F0456092B
:1053F0005A1C0123B6EB511F50F8265003FA02F352
:105400004FEA511703F1FF333DBF50F82720C4F195
:105410002000134003EA05003BBF03FA00F225FA1F
:1054200004F0E0401043F0BD70B57E227F210546B8
:10543000FFF7D8FF18B1012819D0002070BD3E2217
:1054400049212846FFF7CEFF2F2204463121284666
:10545000FFF7C8FF06460134502202365321284682
:10546000B440FFF7BFFF093804FA00F0E6E7302246
:1054700045212846FFF7B6FF01308002DEE7000035
:1054800090F8D63090F8D7201B0403EB026390F815
:10549000D42090F8D500134403EB0020704700009F
:1054A000F8B50F461546044648B905F11F01012617
:1054B000386821F01F01FDF771FE3046F8BD427BD0
:1054C00029463868FDF700FE06460028EDD13B6806
:1054D0006360A368AB4210D213B12068FDF7F0FD02
:1054E000637B28462BB1FDF7E7FD206020B9A06063
:1054F000E3E7FDF7ABFDF8E7A560206805F11F01C4
:10550000012621F01F013860FDF748FE2673D4E71D
:1055100070B50E4602F11F010446154621F01F0129
:105520003046FDF74DFE4CB12168B14206D16068AE
:1055300010B12A46FBF7B8FC0023237370BD0000AE
:10554000F8B50F461446054648B904F11F01012677
:10555000386821F01F01FDF733FE3046F8BD427B6D
:1055600021463868FDF7B0FD06460028EDD1AB684E
:10557000A34210D213B12868FDF7A2FD6B7B204631
:105580002BB1FDF799FD286020B9A860E5E7FDF78C
:105590005DFDF8E7AC60396819B122462868FBF771
:1055A00083FC286804F11F01012621F01F013860E7
:1055B000FDF706FE2E73D0E720B103688B4204BFCF
:1055C000002303737047000010B501390244904274
:1055D00001D1002005E0037811F8014FA34201D06A
:1055E000181B10BD0130F2E7034611F8012B03F838
:1055F000012B002AF9D17047313766656661346145
:10560000653134633430343800000000121000007B
:10561000121100001213000053544D333248373F2B
:105620003F3F0053544D3332483733782F37327869
:105630000053544D3332483734332F3735332F37F7
:105640003530000001105A000310590001205800A5
:1056500003205600100002400800024000080240EB
:1056600000000B002800024008000240040802402D
:1056700006010C00400002400800024008080240F9
:1056800010020D0058000240080002400C080240C1
:1056900016030E00700002400C0002401008024089
:1056A00000040F00880002400C0002401408024071
:1056B00006051000A00002400C000240180802403D
:1056C00010061100B80002400C0002401C08024005
:1056D00016072F0010040240080402402008024070
:1056E0000008380028040240080402402408024050
:1056F000060939004004024008040240280802401C
:10570000100A3A0058040240080402402C080240E3
:10571000160B3B00700402400C04024030080240AB
:10572000000C3C00880402400C0402403408024093
:10573000060D4400A00402400C0402403808024058
:10574000100E4500B80402400C0402403C08024020
:10575000160F460000960000000000000000000048
:105760000000000000000000000000000000000039
:10577000891B0008751B0008B11B00089D1B000851
:10578000A91B0008951B0008811B00086D1B000861
:10579000BD1B000800000000A11C00088D1C0008B3
:1057A000C91C0008B51C0008C11C0008AD1C00087D
:1057B000991C0008851C0008D51C0008000000008A
:1057C000010000000000000063300000C85700081E
:1057D00020290020302B00204172647550696C6FC5
:1057E000740025424F415244252D424C002553451B
:1057F0005249414C2500000002000000000000005A
:10580000C11E0008311F000840004000E043002096
:10581000F043002002000000000000000300000030
:1058200000000000791F00080000000010000000C8
:105830000044002000000000010000000000000003
:105840001C47002001010200E92A0008F92900088C
:10585000952A0008792A00084300000060580008D3
:1058600009024300020100C03209040000010202E3
:105870000100052400100105240100010424020296
:105880000524060001070582030800FF0904010042
:10589000020A00000007050102400000070581021E
:1058A0004000000012000000AC5800081201100176
:1058B00002000040091241570002010203010000EA
:1058C0000403090425424F415244250041746C6190
:1058D000732D436F6E74726F6C0030313233343518
:1058E0003637383941424344454600000000002025
:1058F0000000020002000000000000300000040070
:10590000080000000000002400000800040000005F
:105910000004000000FC0000020000000000043051
:1059200000800000080000000000003800000100B6
:105930000100000000000000D52000088D230008B1
:1059400039240008400040005448002054480020FA
:1059500001000000644800208000000040010000B9
:105960000800000000010000001000000800000016
:105970006D61696E0069646C650000000000802A3A
:1059800000000000AAAAAAAA00000024FFFF00004D
:105990000000000000A00A0000000000000000005D
:1059A000AAAAAAAA00000000FFFF00000000000051
:1059B000000000000000AA0200000000AAAAAAAA93
:1059C00000005500FFFF000000000000CCCC0C00E0
:1059D0002000000000000000AAAAAAAA10000000EF
:1059E000FFFF0000000C000000000000000002406B
:1059F00000000000AAAAAA2A00000140FFFF000040
:105A0000000000000700000050251000000000000A
:105A1000AAA2AAAA50151000FFFF0000000000076C
:105A2000000000000010100000000000AA8AAAAACE
:105A300000101000FFFF0000000000000000000048
:105A40000000000000000000AAAAAAAA00000000AE
:105A5000FFFF0000000000000000000000551105DD
:105A6000E0000000AAAAAAA800011105FFFF00009B
:105A70000000000000000000000000000000000026
:105A8000AAAAAAAA00000000FFFF00000000000070
:105A9000000000000000000000000000AAAAAAAA5E
:105AA00000000000FFFF00000000000000000000F8
:105AB00000000000C1460008C5460008014B000870
:105AC000394E0008954A0008BD4A0008E54A00081A
:105AD0007D4A000800000000CB0400000000000028
:105AE00000001E0000000000FF000000382B002016
:105AF0005C24002000000000185600088304000009
:105B0000235600085004000031560008009600009B
:105B100000000800960000000008000004000000DB
:105B2000C058000800000000000000000000000055
:0C5B300000000000000000000000000069
:00000001FF
